:020000040000FA
:040000006CEF01F0B0
:080008006EEF01F01D52D8A4B7
:100010000BEF00F01200FF0E0000000000000000D7
:1000200000000000000000000000000000000000D0
:1000300000000000000000000000000000000000C0
:1000400000000000000000000000000000000000B0
:1000500000000000000000000000000000000000A0
:100060000000000000000000000000000000FF0F82
:10007000D8A40CEF00F00000000000000000000019
:1000800000000000000000000000000000001D2E25
:100090000BEF00F01200FA0E1D6E06EC00F0FA0EE7
:1000A0001D6E06EC00F0FA0E1D6E06EC00F0FA0E66
:1000B0001D6E06EC00F01C2EEED712000F5257E119
:1000C00018500F6E135223E11150106004D0102805
:1000D000106E196A09D01150106203D0010E196E0A
:1000E00003D01004106E196A1450126004D0122844
:1000F000126E1A6A09D01450126203D0010E1A6EE1
:1001000003D01204126E1A6A1A501914136E1B04CB
:1001100012E10E040AE115501F6E206A1F2AD8B49E
:10012000202A070E1F14156E0CD015041F6E070E23
:100130001F14156E06D0070E1014156E070E12143C
:10014000176E000EEA6E050EE96E1750E926EF38BD
:10015000F00B1F6E000EEA6E050EE96E1550E926D3
:10016000EF501F10166E956A1650836E12000F0422
:100170000F6E1200136A1C6A1C2A13661C901C5214
:10018000FAE112000F0EC16E080E6F6E100E931082
:10019000936E100E81141C6E0D6A100E1C6201D03D
:1001A0000D2A0D5207E1F70E9314936EF70E81148A
:1001B000816E09D0F70E9314936EF70E81141C6EA6
:1001C000080E1C10816E010E056E030E066E020EE7
:1001D000076E060E086E040E096E0C0E0A6E080EEF
:1001E0000B6E090E0C6EC80E116E146E106E126E30
:1001F0001B6A760E186ED59AD588F00ED5141C6E33
:10020000010E1C10D56EF28EF28A010E1C6E4BECA4
:1002100000F0116A146ABAEC00F0010E1C6E4BEC8F
:1002200000F05A0E116EBAEC00F0010E1C6E4BEC91
:1002300000F05A0E146EBAEC00F0100E9310936E8C
:10024000100E81141D6E1E6A100E1D6201D01E2A32
:100250001E500D6E1C6A0D04D8B41C2A1C52EDE110
:10026000010E1B6E170E186E100E9310936E100E6B
:1002700081141C6E1D6A100E1C6201D01D2A1D50B7
:100280000D6E0D52F1E10E5209E1FB0E9314936EC7
:10029000FB0E8114816E010E0E6E0AD0FB0E9314BC
:1002A000936EFB0E81141C6E040E1C10816E0E6A80
:1002B000100E9310936E100E81141D6E1E6A100E98
:1002C0001D6201D01E2A1E500D6E1C6A1C2A0D666E
:1002D0001C901C52EDE1C8D7C2EF00F0EACF01F04C
:1002E000E9CF02F0F4CF03F0F3CF04F0F2A403D08F
:1002F0005EEC00F0F29404C0F3FF03C0F4FF02C010
:08030000E9FF01C0EAFF110052
:020000040030CA
:0E000000240E3F1E008181000FC00FA00F4094
:00000001FF
